:020000040000FA
:0400000057EF00F0C6
:10000800BE4BBE4BBE4BBE4BBE4BBE4BBE4BBE4BA0
:10001800414CBE4BB94CBE4BBE4BBE4BBE4BBE4B10
:10002800BE4BBE4BBE4BBE4BBE4BBE4BBE4B554AEA
:10003800554A554A554A5246BE4BBE4BBE4BBE4B1F
:10004800BE4BBE4BE44ABE4B2B00BE4BBE4BBE4B19
:10005800BE4BBE4BBE4BBE4BBE4BBE4BBE4BBE4B50
:10006800BE4BBE4BBE4BBE4BBE4BBE4BBE4BBE4B40
:10007800BE4BBE4B2B00BE4BBE4BBE4B2B002B00CA
:100088002B002B002B002B002B002B00BE4BBE4B54
:10009800D54ABE4BBE4BBE4B2B002B002B002B0072
:0A00A800BE4BBE4BFF0054EF91F079
:10F75E0000603201022C01CC2F01501701FA1C015E
:10F76E00802501341E014632013033012C3301A8AD
:10F77E002E01C83201C03201383201B83201FE31D9
:10F78E00010A27014C2601EE3101010000000A009A
:10F79E00000064000000E803000010270000A086AF
:10F7AE00010040420F008096980000E1F50500CA66
:10F7BE009A3B010000001000000000010000001044
:10F7CE000000000001000000100000000001000019
:10F7DE00001045724C754D614D654A655665536115
:10F7EE0044690053657074656D62726520004469EA
:10F7FE006D616E636865200056656E64726564693E
:10F80E0020004D657263726564692000446563650E
:10F81E006D62726520004E6F76656D6272652000B6
:10F82E004F63746F62726520004A75696C6C657403
:10F83E0020004665767269657220004A616E7669AF
:10F84E006572200053616D65646920006572726592
:10F85E00757220004A6575646920004D6172646995
:10F86E0020004C756E646920004572726F72200024
:10F87E00417672696C2000416F757420004A75697B
:10F88E006E20004D61727320004D616920002020B2
:10F89E00002054494D4552322066726565206D6FC9
:10F8AE006465202049565420496E746572727570D5
:10F8BE0074204C6F772061766563207469636B3DAD
:10F8CE0038313932B5532031323220626F75636C64
:10F8DE006573203D3E2031736563200D0A002020A4
:10F8EE004370745F54322025356420202043707499
:10F8FE005F54363D25356420204370742049545F93
:10F90E0052424F3D2535642050574D35206F75744A
:10F91E003D20253364202573204541313D25356436
:10F92E0020200D0A20002055415254312048616498
:10F93E007277617265205243363D545820205243EF
:10F94E00373D525820203131353230302C382C4E44
:10F95E002C312020496E746572727570742048695E
:10F96E00676820737572205258200D0A0020546566
:10F97E0073742064697665727320737572203138E2
:10F98E004632374B34322C20493243205254432CCA
:10F99E002050574D2E2E2055415254206574632011
:10F9AE002072657620617672696C20323032312099
:10F9BE000D0A002065783A20553B30333B30333BFF
:10F9CE0032313B31353B31343B30333B23202070D9
:10F9DE006F7572203033206D617273203230323188
:10F9EE00202C20313548313420204D6572637265EC
:10F9FE006469200D0A0020553B32343B30383B31D0
:10FA0E00373B31383B33363B3034232020706F7513
:10FA1E007220323420416F757420323031372020FD
:10FA2E0031384833362030343D4A657564690D0AE5
:10FA3E000D0A0020496E69742052544320466F729D
:10FA4E0063656520612073616D6564692030322FB6
:10FA5E0030332F32312031383A34363A353720763A
:10FA6E00696120205242313D30200D0A00204E4364
:10FA7E004F204E756D65726963616C20436F6E74B5
:10FA8E00726F6C6C6564204F7363696C6C61746526
:10FA9E007572203A20536F727469652073757220E7
:10FAAE00524332200D0A0020456E74726565204166
:10FABE0044432045413120313220626974732073F2
:10FACE007572205241312020706F757220636F6EF7
:10FADE007369676E652050574D35200D0A00204D15
:10FAEE006F64756C652050573520314B687A202035
:10FAFE00313020626974732C20286C69E920E02073
:10FB0E00544D52342029202C736F72746965205223
:10FB1E0043350D0A000D0A2052617070656C206627
:10FB2E006F726D617420646520636465203A2022D3
:10FB3E00553B4A4A3B4D4D3B41413B48483B4D4D61
:10FB4E003B6A533B2322200D0A00207573616765C3
:10FB5E0020646520534D543120636F6D707465754C
:10FB6E00722032346269747320706F75722063680C
:10FB7E00726F6E6F6D6574726167650D0A00204954
:10FB8E006E6974204E434F3120463D31304B687ABA
:10FB9E002020553D2533642020483D253364204CDC
:10FBAE003D25336420736F697420305825303658E4
:10FBBE0020002052652D4C65637475726520657446
:10FBCE0020616666696368616765206465732037C6
:10FBDE0020526567697374726573204453333233F0
:10FBEE0031200D0A0020436F6D70696C65206C65C5
:10FBFE002025732061202573205554430D0A206162
:10FC0E007665632076657273696F6E20584338206F
:10FC1E003A202025640D0A002048617264776172D3
:10FC2E0065203A20424153452031384632374B3415
:10FC3E00322020464F534320696E7465726E6520E4
:10FC4E003D36344D487A200D0A00204D414A20524F
:10FC5E0054432076696120554152543120617665B6
:10FC6E006320525820495654204869676820496ECF
:10FC7E0074657272757074200D0A00205465737469
:10FC8E002050726573656E6365204932432064654A
:10FC9E007669636520286164726573736167652098
:10FCAE00382062697473290D0A002052544320448F
:10FCBE00533332333120737572206C652062757345
:10FCCE002049324331205243333D53434C2052435B
:10FCDE00343D5344410D0A00204020646563696D34
:10FCEE00616C20232534752020736F697420404485
:10FCFE0065766963653762697473203D20305825D7
:10FD0E00303258200020537461727420534D543198
:10FD1E0020706F75722031206D657375726520418C
:10FD2E0044432031322062697473200D0A0020464C
:10FD3E006F72E761676520446174652065742048C1
:10FD4E006575726520525443207669612050696E44
:10FD5E00205242310D0A002050726F6A6574204D98
:10FD6E00504C414258203A204956545F54657374A2
:10FD7E005F31384632374B3432200D0A0020535152
:10FD8E004135302073796E6368726F20416E616CFD
:10FD9E0079736572202073757220524133200D0ADB
:10FDAE00002053746F7020534D54312020204E622A
:10FDBE002054696373206176656320756C746F617E
:10FDCE00202D3E20000D0A457272657572207375E6
:10FDDE0072204A6F75722053656D61696E65206A77
:10FDEE00532E200D0A0020496E6974204D79204152
:10FDFE0044432031326269747320656E7472656596
:10FE0E00204541310D0A0020536F727469652046FA
:10FE1E004F53432F342031364D487A20737572205C
:10FE2E00524136200D0A00546573742049565420F1
:10FE3E00696E74657272757074202031384632376F
:10FE4E004B34320D0A0020536F72746965204E4395
:10FE5E004F312031304B687A207375722052433205
:10FE6E00200D0A00202331204163746976652073CA
:10FE7E006F72746965205351573D31487A3A200D9F
:10FE8E000A0020496E69742050574D35206F7574E5
:10FE9E0020524335203D203235250D0A0045637230
:10FEAE006974757265204453333233312E2E2E20F1
:10FEBE004F4B0D0A002054494D455234207469634E
:10FECE006B733D3634B553200D0A000D0A2048657C
:10FEDE006C7020436F6D6D616E646573203A0D0A10
:10FEEE0000504346383537344120386269747320E8
:10FEFE00492F4F00504346383537342038626974E5
:10FF0E007320492F4F004C43442032313139203277
:10FF1E0078313663617273003031323334353637AF
:10FF2E00383941424344454600204574617420707F
:10FF3E00696E20524231203D2000202C20736F69C3
:10FF4E00742020256C7520755300454550524F4D39
:10FF5E00203531326279746573000D0A204D414AA5
:10FF6E0020525443200D0A004144584C333435205E
:10FF7E00626F61726400204D414A2052544320202A
:10FF8E000D0A004F4C454420535344313330360054
:10FF9E006E6F6E20726563656E73E9002052656741
:10FFAE0069737472652023004170722031362032DD
:10FFBE003032310052544320445333323331002017
:10FFCE0048656C70200D0A0052656375203A0D0A63
:10FFDE000030393A35333A303500286E756C6C295D
:10FFEE000020474F0D0A00206F6B0D0A00202500E0
:01FFFE000002
:020000040001F9
:10000000600E3901D96F000EDB6F000EDD6F080E38
:10001000DF6F000EDE6F67EC8FF0C5EC97F0D6EC6B
:1000200097F023EC98F0F6EC97F01DEC96F075EC59
:1000300098F005EC98F036EC99F0D1EC94F068EC7F
:1000400097F0410E9EEC99F0420E9EEC99F0430E13
:100050009EEC99F00D0E9EEC99F00A0E9EEC99F034
:10006000000E436E020E446E000E366EE4EC96F007
:10007000650E1C6EFD0E1D6EDEEC93F043C0ECF0C1
:1000800044C0EDF0F30E0001EE6FFB0EEF6FB60E05
:10009000F06FFF0EF16FDF0EF26FFF0EF36F090EC0
:1000A000F56F100EF46FEDEC84F043C01CF044C00B
:1000B0001DF032EC94F07B0E1C6EF90E1D6EDEEC22
:1000C00093F0260E1C6EFC0E1D6EDEEC93F0340ECB
:1000D0001C6EF90E1D6EDEEC93F09F0E1C6EF80E7A
:1000E0001D6EDEEC93F0B50E1C6EFA0E1D6EDEEC8E
:1000F00093F0C30E1C6EFE0E1D6EDEEC93F0EC0E44
:100100001C6EFA0E1D6EDEEC93F0540E1C6EFE0E8D
:100110001D6EDEEC93F08B0E1C6EFD0E1D6EDEEC84
:1001200093F0150E1C6EFE0E1D6EDEEC93F07B0E32
:100130001C6EFA0E1D6EDEEC93F0580E1C6EFB0E5C
:100140001D6EDEEC93F0B80E1C6EFC0E1D6EDEEC28
:1001500093F03C0E1C6EFD0E1D6EDEEC93F0580EFF
:100160001C6EFC0E1D6EDEEC93F0A30E0101EC6F15
:10017000570EEB6F020EE82EFED7EB2FFCD7EC2FBD
:10018000FAD700F0000E0001B26F000EB16F000E42
:10019000B06F000EAF6F000EAE6F000EAD6F900E21
:1001A0001C6EFE0E1D6EDEEC93F075EC98F0000EEA
:1001B0001D6EFA0E1C6E38EC96F0E4EC96F03901E8
:1001C000949BBA863F013E9F000E3A6F000E396F36
:1001D000000E386FBA96D70E3B6FA30E3C6F000E21
:1001E0003D6F43C0ECF044C0EDF08C0E0001EE6FAB
:1001F000FB0EEF6F6F00F4FCF0F0F16B6F00F0FCA2
:10020000F2F0F36B6F00ECFCF4F0F56B6F00ECFCBC
:10021000F6F06F00F0FCF7F06F00F4FCF8F0EDEC96
:1002200084F043C01CF044C01DF032EC94F0E4ECC8
:1002300096F03F013E8FE4EC96F0B2EC93F0AC8E7A
:10024000948EF40E1C6EFD0E1D6EDEEC93F023EC0E
:1002500098F0000E0001B76F000EB86F000EB96F76
:10026000000EBA6FB70EA96F000EAA6F000EB76F1F
:10027000000EB86F000EB96F000EBA6F000EAC6FB3
:10028000000EAB6F130E1C6EFD0E1D6EDEEC93F0B8
:100290003F01208B1F8F3E01F881F8B152EF81F0B2
:1002A00054EF81F04DEF81F0F0510101EC6FEB6BF9
:1002B0003E01EF510101EB250001AB6F3E01000E45
:1002C0000101EC210001AC6F3F011F9F000E436E46
:1002D000020E446EE5EC98F01CC0B7F01DC0B8F0FB
:1002E0001EC0B9F01FC0BAF0AF0E1C6EFD0E1D6E21
:1002F000DEEC93F043C0ECF044C0EDF0B7C0EEF09C
:10030000B8C0EFF0B9C0F0F0BAC0F1F0000E0001D3
:10031000F36F0A0EF26F84EC8AF043C01CF044C005
:100320001DF032EC94F043C0ECF044C0EDF0480E08
:100330000001EE6FFF0EEF6FB7C0EBF1B8C0ECF14C
:10034000B9C0EDF1BAC0EEF1070EADEF81F00101D9
:10035000D890EE33ED33EC33EB33E82EA7EF81F09A
:10036000EBC1F0F0ECC1F1F0EDC1F2F0EEC1F3F051
:10037000EDEC84F043C01CF044C01DF032EC94F06E
:10038000E4EC96F0000E436E020E446E60000FF136
:10039000D9FF600013F1DAFF000EDF6EE4EC96F097
:1003A000890E1C6EFC0E1D6EDEEC93F03D017599FE
:1003B000738F000E346E020E336E345009E1FE0E60
:1003C000335CD8A0E6EF81F0E8EF81F0EAEF81F04E
:1003D000C8EF82F033C01CF034C01DF06BEC96F017
:1003E0000009D8B4F6EF81F0F8EF81F0C0EF82F0A9
:1003F000D89034300101EB6F33302F6EEBC130F009
:1004000043C0ECF044C0EDF0E60E0001EE6FFC0ED0
:10041000EF6F33C0F0F034C0F1F02FC0F2F030C015
:10042000F3F0EDEC84F075EF82F043C01CF044C0B3
:100430001DF0020E1E6EFF0E1F6E89EC92F0B8EFDB
:1004400082F043C01CF044C01DF0140E1E6EFF0E5F
:100450001F6E89EC92F0B8EF82F043C01CF044C0EC
:100460001DF0EF0E1E6EFE0E1F6E89EC92F0B8EFBF
:1004700082F043C01CF044C01DF0910E1E6EFF0EB2
:100480001F6E89EC92F0B8EF82F043C01CF044C0BC
:100490001DF0760E1E6EFF0E1F6E89EC92F0B8EF07
:1004A00082F043C01CF044C01DF0580E1E6EFF0EBB
:1004B0001F6E89EC92F0B8EF82F043C01CF044C08C
:1004C0001DF0C20E1E6EFF0E1F6E89EC92F0B8EF8B
:1004D00082F043C01CF044C01DF09E0E1E6EFF0E45
:1004E0001F6E89EC92F0B8EF82F02FC0EBF130C0B4
:1004F000ECF10101EC51000AD8B481EF82F069EF10
:1005000082F0EB51270AD8B415EF82F00F0AD8B465
:1005100015EF82F0010AD8B415EF82F0030AD8B4BF
:1005200015EF82F01D0AD8B421EF82F00F0AD8B47B
:100530002DEF82F0010AD8B42DEF82F0030AD8B46F
:100540002DEF82F0010AD8B42DEF82F0070AD8B45B
:1005500039EF82F06F0AD8B445EF82F0040AD8B4BC
:1005600051EF82F03F0AD8B45DEF82F069EF82F07C
:1005700043C01CF044C01DF032EC94F0E4EC96F063
:10058000020E3324336E000E3420346EDDEF81F022
:100590003D01739F7589E4EC96F0350E1C6EFE0EDE
:1005A0001D6EDEEC93F03901938794859981908FCD
:1005B000D28ED28C720E1C6EFE0E1D6EDEEC93F08F
:1005C000EF0E1C6EFF0E1D6EDEEC93F0400E01016F
:1005D000806F0E0E0001E36F80C1E4F0680ED9EC6D
:1005E00091F0F50E1C6EFF0E1D6EDEEC93F0090E01
:1005F0000101EC6F1E0EEB6FE40EE82EFED7EB2F21
:10060000FCD7EC2FFAD700F0000E346E010E336EDB
:10061000345009E1200E335CD8A011EF83F013EFC2
:1006200083F015EF83F021EF83F0800E3324D96E31
:10063000010E3420DA6E000EDF6E334A342A08EFE2
:1006400083F0370E1C6EFF0E1D6EDEEC93F0CB5068
:10065000020B300F68EC98F0E4EC96F0CBB233EF7D
:1006600083F035EF83F060EF83F0410E1C6EFA0EDD
:100670001D6EDEEC93F0000E0101806F570E816F4E
:10068000160E826F180E836F060E846F020E856F32
:10069000030E866F210E876F000E886FBA86800E5C
:1006A000296E010E2A6E29C0E3F02AC0E4F0000E84
:1006B0000001E66F080EE56F680EF5EC92F0BA9651
:1006C000520E0101EC6F2B0EEB6F000EE82EFED7E1
:1006D000EB2FFCD7EC2FFAD700F0C00E1C6EFB0EF0
:1006E0001D6EDEEC93F0000E326E000E316EAA0E1F
:1006F0001C6EFF0E1D6EDEEC93F03150300F9EEC41
:1007000099F0090E9EEC99F0010E0001E66F315050
:10071000F5EC94F00001B46FE4EC96F0314A322A23
:10072000325009E1080E315CD8A099EF83F09BEFBD
:1007300083F077EF83F0E4EC96F0EAEC89F0520E68
:100740000101EC6F2B0EEB6F000EE82EFED7EB2FA6
:10075000FCD7EC2FFAD700F0000E326E000E316E8F
:1007600010EC91F0520E0101EC6F2B0EEB6F000EAE
:10077000E82EFED7EB2FFCD7EC2FFAD700F036048B
:10078000D8A4C5EF83F0C7EF83F078EF84F0390188
:100790009397D60E1C6EFF0E1D6EDEEC93F0000ECE
:1007A0001C6E010E1D6E32EC94F0E4EC96F0000E1F
:1007B000276E010E286E60009FF0D9FF6000A3F045
:1007C000DAFF550EDE18D8A4E8EF83F0EAEF83F0E5
:1007D00016EF84F020EE01F02750D9262850DA22B7
:1007E0003B0EDE18D8A4F7EF83F0F9EF83F016EF95
:1007F00084F020EE13F02750D9262850DA223B0E41
:10080000DE18D8A406EF84F008EF84F016EF84F029
:10081000680E1C6EFF0E1D6EDEEC93F0F7EC88F098
:10082000E4EC96F0000E276E000E286E60009FF03C
:10083000D9FF6000A3F0DAFF480EDE18D8A423EF3A
:1008400084F025EF84F076EF84F020EE01F027505D
:10085000D9262850DA22650EDE18D8A432EF84F0AB
:1008600034EF84F076EF84F020EE02F02750D926A2
:100870002850DA226C0EDE18D8A441EF84F043EF42
:1008800084F076EF84F020EE03F02750D92628502C
:10089000DA22700EDE18D8A450EF84F052EF84F004
:1008A00076EF84F0D90E1C6EFE0E1D6EDEEC93F01A
:1008B000840E1C6EFF0E1D6EDEEC93F0C10E1C6EDE
:1008C000F90E1D6EDEEC93F0CD0E1C6EFF0E1D6E4C
:1008D000DEEC93F0000E1C6E010E1D6E32EC94F0F7
:1008E000E4EC96F0000E276E000E286E3901938717
:1008F0003E01F881F8B17FEF84F081EF84F07AEF68
:1009000084F0F0510101EC6FEB6B3E01EF510101FE
:10091000EB250001AB6F3E01000E0101EC2100014F
:10092000AC6FFF0EB1152F6E030EB215306EBA8686
:100930002FC01CF030C01DF038EC96F0010E31ECE9
:100940008CF0BA9643C0ECF044C0EDF0EC0E000120
:10095000EE6FF80EEF6FB1C0F0F0B2C0F1F0AFC0C3
:10096000F2F0B0C0F3F0ADC0F4F0AEC0F5F02FC0BF
:100970001CF030C01DF0000E1F6E0A0E1E6E16EC2D
:1009800092F01CC0F6F01DC0F7F0FB0E0001F86FEE
:10099000FF0EF96FABC0FAF0ACC0FBF0EDEC84F0E9
:1009A00043C01CF044C01DF032EC94F0314A322AAE
:1009B000325009E13D0E315CD8A0E1EF84F0E3EF65
:1009C00084F0B0EF83F0000E326E000E316EE4EC76
:1009D00096F0B0EF83F057EF00F0F00E0101E16FF9
:1009E000000EE26FD6EF88F0250EEA19D8B4FBEFBF
:1009F00084F0FDEF84F00BEF85F06000B3F3D9FFD6
:100A00006000B7F3DAFF6000ABF7DFFF0001EC4BEB
:100A1000ED2BD6EF88F0000EE96F000EE86F000EA8
:100A2000E76F18EF85F00101E7850001EE4BEF2B32
:100A30006000BBF3F6FF6000BFF3F7FF000EF86E37
:100A40000800F550300AD8B413EF85F028EF85F090
:100A50006000BBF3F6FF6000BFF3F7FF000EF86E17
:100A60000800F55052EC96F0D8A039EF85F03BEF36
:100A700085F03DEF86F0000E0101E96F000EE86F92
:100A8000E8C11CF0E9C11DF0000E1F6E0A0E1E6EBB
:100A90003FEC97F01CC0E8F11DC0E9F1D00E000159
:100AA000FC6FFF0EFD6F6000BBF3F6FF6000BFF34D
:100AB000F7FF000EF86E0800F550FE6FFF6BFC515B
:100AC000FE27FD51FF23FE510101E8270001FF51E0
:100AD0000101E9230001EE4BEF2B6000BBF3F6FFB1
:100AE0006000BFF3F7FF000EF86E0800F55052ECFF
:100AF00096F0D8B07EEF85F080EF85F040EF85F07E
:100B00003DEF86F0E7893DEF86F0E78F70EF86F0E6
:100B1000600087F7D9FF60008BF7DAFF6F0078FF7E
:100B2000DDF16F0074FFDEF1020EE127000EE2231B
:100B3000DD51DE11D8A49FEF85F0A1EF85F0A5EF80
:100B400085F0E80EDD6FFF0EDE6F000EE06F000E29
:100B5000DF6FAEEF85F00101DF4BE02BDF51DD25CC
:100B60000001FC6F0101E051DE210001FD6F60001A
:100B7000F3F3F6FF6000F7F3F7FF000EF86E1F0EB9
:100B8000F76403D00800F55007D06F00DBFFE9FFE2
:100B90006F00DFFFEAFFEF500009D8A4D2EF85F025
:100BA000D4EF85F0ABEF85F00101E851DF5DE9514D
:100BB000E059D8B0DEEF85F0E0EF85F0E6EF85F0A4
:100BC000DF51E85FE051E95BF7EF85F0000EE96F78
:100BD000000EE86FF7EF85F06000B3F3D9FF600017
:100BE000B7F3DAFF200EDF6E0001EC4BED2B0101B5
:100BF000E807D8A0E907E82906E1E929D8A403EF26
:100C000086F005EF86F0ECEF85F029EF86F06000C6
:100C100077F7F6FF60007BF7F7FF000EF86E6000D5
:100C2000B3F3D9FF6000B7F3DAFF1F0EF76403D008
:100C30000800F55007D06F00DBFFE9FF6F00DFFF12
:100C4000EAFFEF50DF6E0101DD4BDE2B0001EC4BC4
:100C5000ED2B0101DF07D8A0E007DF2906E1E0293D
:100C6000D8A435EF86F037EF86F007EF86F0D6EFA1
:100C700088F0C00EE71370EF86F06000BBF3F6FF5C
:100C80006000BFF3F7FF0001EE4BEF2B000EF86E94
:100C900008006F00D4FFEAF10101EA51000AD8B45C
:100CA000EEEF88F0580AD8B485EF85F03C0AD8B446
:100CB00070EF86F00D0AD8B470EF86F0050AD8B44C
:100CC00082EF85F01F0AD8B488EF85F0060AD8B401
:100CD00039EF86F00D0AD8B485EF85F0D6EF88F0AD
:100CE000E7C1FCF0C00E0001FC17D8A47AEF86F033
:100CF0007CEF86F0C4EF86F00101E7A982EF86F071
:100D000084EF86F09CEF86F0600087F7D9FF6000E3
:100D10008BF7DAFF6F0078FFE3F16F0078FFE4F103
:100D20006F0078FFE5F16F0078FFE6F1040EE12730
:100D3000000EE223B1EF86F0600087F7D9FF600074
:100D40008BF7DAFF6F0078FFE3F16F0074FFE4F1D7
:100D5000000EE4BFFF0EE56FE66F020EE127000E06
:100D6000E223E6BFB8EF86F0B6EF86F058EF87F0E3
:100D7000030EE713E61FE51FE41FE36D000EE423F7
:100D8000E523E62358EF87F00101E7A9CAEF86F0D3
:100D9000CCEF86F0E4EF86F0600087F7D9FF6000C3
:100DA0008BF7DAFF6F0078FFE3F16F0078FFE4F173
:100DB0006F0078FFE5F16F0078FFE6F1040EE127A0
:100DC000000EE22358EF87F0600087F7D9FF60003C
:100DD0008BF7DAFF6F0078FFFCF06F0074FFFDF017
:100DE000FCC0E3F1FDC0E4F1E56BE66B020EE12728
:100DF000000EE22358EF87F0010EEA6FEA51040D6E
:100E0000980EF324F66EF70EF420F76EF86A000ED3
:100E1000F8220900F550E35D0900F550E459090096
:100E2000F550E5590900F550E659D8B01AEF87F0AA
:100E30001CEF87F01EEF87F068EF87F0EA2B0A0EB1
:100E4000EA19D8A426EF87F028EF87F0FEEF86F0A6
:100E500068EF87F0010EEA6FEA51040DC00EF3242B
:100E6000F66EF70EF420F76EF86A000EF82209000D
:100E7000F550E35D0900F550E4590900F550E559D6
:100E80000900F550E659D8B048EF87F04AEF87F0EF
:100E90004CEF87F068EF87F0EA2B080EEA19D8A428
:100EA00054EF87F056EF87F02CEF87F068EF87F06C
:100EB000E751C00B000AD8B4FCEF86F0800AD8B422
:100EC0002AEF87F0400AD8B4FCEF86F068EF87F08D
:100ED000E851E911D8B46FEF87F071EF87F081EF37
:100EE00087F0E7C1FCF0030E0001FC17D8B47BEFDC
:100EF00087F07DEF87F081EF87F00101E807D8A048
:100F0000E9070101EA510001FC6FFD6B0101E851A5
:100F10000001FC5DFD51800AFE6F0101E951800A6C
:100F20000001FE59D8B097EF87F099EF87F0A0EF56
:100F300087F00101EA51E85F000EE95BA5EF87F059
:100F4000000E0101E96F000EE86FE7A5AAEF87F038
:100F5000ACEF87F0E6EF87F0E7C1FCF0030E00018D
:100F6000FC17D8B4B6EF87F0B8EF87F0C2EF87F080
:100F70006000B3F3D9FF6000B7F3DAFF2D0EDF6E28
:100F8000EC4BED2B0101E851E911D8B4CAEF87F021
:100F9000CCEF87F01DEF88F06000B3F3D9FF60005D
:100FA000B7F3DAFF300EDF6E0001EC4BED2B0101E1
:100FB000E807D8A0E907E851E911D8A4E2EF87F0E3
:100FC000E4EF87F0CCEF87F01DEF88F0E851E911EE
:100FD000D8B4EDEF87F0EFEF87F007EF88F060000F
:100FE000B3F3D9FF6000B7F3DAFF200EDF6E000124
:100FF000EC4BED2B0101E807D8A0E907E851E91116
:10100000D8A405EF88F007EF88F0EFEF87F0E7C18D
:10101000FCF0030E0001FC17D8B411EF88F013EFB9
:1010200088F01DEF88F06000B3F3D9FF6000B7F3DC
:10103000DAFF2D0EDF6EEC4BED2BEAC1DBF1010187
:10104000DC6BC8EF88F0DBC1FCF0DCC1FDF0000117
:10105000D890FC37FD37D890FC37FD37980EFC252B
:10106000F66EF70EFD21F76EF86A000EF822090001
:101070006F00D4FF20F009006F00D4FF21F00900B9
:101080006F00D4FF22F00A006F00D4FF23F0E3C109
:101090001CF0E4C11DF0E5C11EF0E6C11FF02AEC12
:1010A0008EF01CC0E4F01DC0E5F01EC0E6F01FC0CD
:1010B000E7F00A0E0001E86F000EE96F000EEA6F1C
:1010C000000EEB6F86EC90F00001E451300F01014F
:1010D000EA6FBCEF88F0E3C11CF0E4C11DF0E5C18C
:1010E0001EF0E6C11FF0DBC1FCF0DCC1FDF0000129
:1010F000D890FC37FD37D890FC37FD37C00EFC2563
:10110000F66EF70EFD21F76EF86A000EF822090060
:101110006F00D4FF20F009006F00D4FF21F0090018
:101120006F00D4FF22F00A006F00D4FF23F02AECF6
:101130008EF01C500F0B0101DA6F260EDA25F66EC9
:10114000F76AFF0EF722F86A000EF82208006F0017
:10115000D4FFEAF1BCEF88F0E751C00B000AD8B425
:1011600023EF88F0800AD8B46BEF88F0400AD8B437
:1011700023EF88F0BCEF88F06000B3F3D9FF600084
:10118000B7F3DAFF6000ABF7DFFF0001EC4BED2BAC
:101190000101DB07D8A0DC07DB2906E1DC29D8A4A4
:1011A000D4EF88F0D6EF88F0ACEF88F06000BBF3A6
:1011B000F6FF6000BFF3F7FF0001EE4BEF2B000ED0
:1011C000F86E08006F00D4FFEAF10101EA51D8A4DB
:1011D000ECEF88F0EEEF88F0F4EF84F06000B3F30A
:1011E000D9FF6000B7F3DAFF000EDF6E1200000EC9
:1011F0000001EA6F020EE96F000EEC6F000EEB6F5C
:10120000000E2D24D96E010E2E20DA6E000EDF6E38
:101210002E5007E1160E2D5CD8B011EF89F013EFB8
:1012200089F0DDEF89F02E5009E1130E2D5CD8A076
:101230001CEF89F01EEF89F0DDEF89F0000EEE6FF4
:10124000020EED6F57EF89F0000EED25D96E010EFD
:10125000EE21DA6E3B0EDE18D8A431EF89F033EFC1
:1012600089F055EF89F0000EED25D96E010EEE21C3
:10127000DA6E000EDF6E000EE9251C6E010EEA210B
:101280001D6E16EC8BF0940E0001EB25D96E000E4E
:10129000EC21DA6E600073F0DFFFEB4BEC2B010EFC
:1012A000ED25E96F000EEE21EA6FED4BEE2B2D5090
:1012B000ED5D2E50EE59D8A060EF89F062EF89F015
:1012C00024EF89F0000EE9251C6E010EEA211D6E47
:1012D00016EC8BF0940E0001EB25D96E000EEC217C
:1012E000DA6E600073F0DFFF94C03EF095511F0B83
:1012F0003D6E96C03CF097C040F098C041F09951C7
:10130000070B3F6E3D50EEEC98F01C503B6E0C0E00
:101310003B648DEF89F08FEF89F091EF89F0000E3B
:101320003B6E070E3F6497EF89F099EF89F0A1EFCC
:1013300089F0000E3F6ED30E1C6EFD0E1D6EDEECAE
:1013400093F0000E0101806F000E426E42C081F1E9
:101350004150E5EC95F00101826F4050E5EC95F0CD
:101360000101836F3FC084F13E50E5EC95F001012F
:10137000856F3D50E5EC95F00101866F3C50E5EC42
:1013800095F00101876F000E886F800E296E010EA7
:101390002A6E29C0E3F02AC0E4F0000E0001E66FD7
:1013A000080EE56F680EF5EC92F0AB0E1C6EFE0EAB
:1013B0001D6EDEEC93F0E9EF89F0230E1C6EFB0E40
:1013C0001D6EDEEC93F0040E1C6EFA0E1D6EDEEC4C
:1013D00093F01200CCEC8EF0000E0001CC6FD60E14
:1013E0001C6E000E1D6E3E5018EC95F02F0E000185
:1013F000D86FD90E1C6E000E1D6E3D5018EC95F086
:101400002F0E0001DB6FDC0E1C6E000E1D6E3C50BB
:1014100018EC95F0000E0001DE6F000E0201806FE7
:101420003F50020DBB0EF324D96E000EF420DA6E8D
:101430006F0078FF1CF06F0074FF1DF0DEEC93F07E
:10144000200E68EC98F0800E1C6E020E1D6E3E5051
:1014500018EC95F0800E1C6E020E1D6E32EC94F0AE
:10146000200E68EC98F03D50EEEC98F01C503B6E6E
:101470003B50020DC00EF324D96E010EF420DA6E3B
:101480006F0078FF1CF06F0074FF1DF0DEEC93F02E
:10149000200E68EC98F0800E1C6E020E1D6E3C5003
:1014A00018EC95F0800E1C6E020E1D6E32EC94F05E
:1014B000200E68EC98F0CC0E1C6E000E1D6E405095
:1014C00018EC95F0480E0001CE6FCF0E1C6E000E8A
:1014D0001D6E415018EC95F04D0E0001D16FD20EEB
:1014E0001C6E000E1D6E425018EC95F0530E00015C
:1014F000D46F000ED56FCC0E1C6E000E1D6E32EC3C
:1015000094F0E4EC96F01200EEC0F4F0EFC0F5F0C9
:10151000F0C0F6F0F1C0F7F0F4C01CF0F5C01DF01B
:10152000F6C01EF0F7C01FF0F2C020F0F3C021F0AB
:10153000000E21BEFF0E226E236E2AEC8EF01CC020
:10154000F4F01DC0F5F01EC0F6F01FC0F7F000016A
:10155000EC4BED2BF451F511F611F711D8A4B3EFC4
:101560008AF0B5EF8AF08CEF8AF06000B3F3D9FF10
:101570006000B7F3DAFF000EDF6EEC07D8A0ED07CE
:10158000EEC0E4F0EFC0E5F0F0C0E6F0F1C0E7F047
:10159000F2C0E8F0F3C0E9F0000EE9BFFF0EEA6F19
:1015A000EB6F86EC90F00001E451F86FEEC01CF098
:1015B000EFC01DF0F0C01EF0F1C01FF0F2C020F02F
:1015C000F3C021F0000E21BEFF0E226E236E2AEC26
:1015D0008EF01CC0EEF01DC0EFF01EC0F0F01FC07A
:1015E000F1F0090E0001F865F8EF8AF0FAEF8AF0E1
:1015F000FCEF8AF0070EF827300EF8276000B3F3EF
:10160000D9FF6000B7F3DAFF6000E3F3DFFFEC0718
:10161000D8A0ED07EE51EF11F011F111D8A413EF9E
:101620008BF015EF8BF0C0EF8AF012001AEF8BF001
:101630001C4A1D2A600073F0D9FF600077F0DAFFC2
:10164000200EDE18D8B427EF8BF029EF8BF018EFBF
:101650008BF0600073F0D9FF600077F0DAFF090EBD
:10166000DE18D8B436EF8BF038EF8BF018EF8BF034
:10167000000E216E000E206E600073F0D9FF600036
:1016800077F0DAFF2D0EDE18D8A449EF8BF04BEF80
:101690008BF050EF8BF0202A1C4A1D2A73EF8BF041
:1016A000600073F0D9FF600077F0DAFF2B0EDE18D0
:1016B000D8A45DEF8BF05FEF8BF073EF8BF01C4ADB
:1016C0001D2A73EF8BF0600073F0D9FF600077F094
:1016D000DAFFDF501E6E21500A0DF3501E24D00F8A
:1016E000216E5FEF8BF0600073F0D9FF600077F040
:1016F000DAFF2F0EDF647FEF8BF081EF8BF08FEF3F
:101700008BF0600073F0D9FF600077F0DAFF390EDC
:10171000DF648DEF8BF08FEF8BF063EF8BF0205059
:10172000D8B495EF8BF097EF8BF0A4EF8BF02150AE
:101730001E6E1F6A1E1E1F1E1E4A1F2A1EC01CF080
:101740001FC01DF0A7EF8BF021C01CF01D6A120016
:10175000A4EC98F00009D8B4B0EF8BF0B2EF8BF0A6
:10176000E4EF8BF0BFEF8BF023EC99F030EF8CF0CF
:1017700098EC99F030EF8CF0000E30EF8CF078C0E0
:101780000CF079C00DF020EE69F002D8D2EF8BF0AA
:101790000500FA6EDE50FD6EDE50FE6EDE50FF6E0E
:1017A000FA501200010AD8B4BCEF8BF0030AD8B487
:1017B000B4EF8BF0010AD8B4B8EF8BF0070AD8B4B5
:1017C000BCEF8BF0BCEF8BF099EC98F00009D8B42B
:1017D000ECEF8BF0EEEF8BF02FEF8CF000018951E6
:1017E000030B0009D8B4F7EF8BF0F9EF8BF005EF9E
:1017F0008CF0010E0E6E8951030B0F6E0E500F5EB2
:1018000089510F18FC0B0F18896F60000FF2D9FF78
:10181000600013F2DAFFDF50106E834B842B8507D4
:10182000D8A0860785518611D8A419EF8CF01BEF3C
:101830008CF023EF8CF0C0EC92F00E6E0E50126E16
:10184000136A27EF8CF0000E136E030E126E12C097
:1018500011F0105045EC99F0115030EF8CF0030E60
:1018600012000001EF6FCCEC8EF0000E0001CC6F87
:10187000000ED66FCC0E1C6E000E1D6E405018EC84
:1018800095F0480E0001CE6FCF0E1C6E000E1D6E3F
:10189000415018EC95F04D0E0001D16FD20E1C6E28
:1018A000000E1D6E425018EC95F0530E0001D46FDF
:1018B000000ED56FD60E1C6E000E1D6E3E5018EC3D
:1018C00095F02F0E0001D86FD90E1C6E000E1D6E04
:1018D0003D5018EC95F02F0E0001DB6FDC0E1C6EF6
:1018E000000E1D6E3C5018EC95F0000E0001DE6FEE
:1018F0003D50EEEC98F01C503B6E4250EEEC98F0F0
:101900001C503A6E0001EF05D8A489EF8CF08BEFE4
:101910008CF0A3EF8CF0D60E1C6E000E1D6E32EC18
:1019200094F09C0E1C6EF80E1D6EDEEC93F0CC0E47
:101930001C6E000E1D6E32EC94F09C0E1C6EF80EA8
:101940001D6EDEEC93F012003901A3A7AAEF8CF014
:10195000ACEF8CF013EF8DF093A7B1EF8CF0B3EFF9
:101960008CF013EF8DF06F00A0F738F00D0E3818E3
:10197000D8B4BDEF8CF0BFEF8CF0CAEF8CF02C50D8
:1019800009E1800E2B5CD8A0C8EF8CF0CAEF8CF078
:10199000EEEF8CF0010E366EA3A7D1EF8CF0D3EFF3
:1019A0008CF0DCEF8CF0000E2B24D96E010E2C2075
:1019B000DA6E6F00A3F7DFFF000E2B24D96E010E45
:1019C0002C20DA6E000EDF6E2BC02DF02CC02EF016
:1019D000000E2C6E000E2B6E13EF8DF0000E2B24DC
:1019E000D96E010E2C20DA6E6000E3F0DFFF2B4A87
:1019F0002C2A2BC02DF02CC02EF0A3A702EF8DF0C7
:101A000004EF8DF013EF8DF0000E2B24D96E010E34
:101A10002C20DA6E6F00A3F7DFFF2B4A2C2A2BC095
:101A20002DF02CC02EF01100000E216E1FBE1DEFF8
:101A30008DF01BEF8DF023EF8DF01E6C1F1ED8B0C4
:101A40001F2A010E216E1DBE2AEF8DF028EF8DF0AA
:101A500030EF8DF01C6C1D1ED8B01D2A010E211A0E
:101A6000000E236E000E226E1E501F10D8B43BEFE6
:101A70008DF03DEF8DF065EF8DF0010E206E45EF9E
:101A80008DF0D8901E361F36202A1FAE4AEF8DF0FB
:101A90004CEF8DF041EF8DF0D890223623361E505A
:101AA0001C5C1F501D58D8A058EF8DF05AEF8DF0D8
:101AB0005FEF8DF01E501C5E1F501D5A2280D89083
:101AC0001F321E32202E4CEF8DF02150D8B46BEF18
:101AD0008DF06DEF8DF071EF8DF0226C231ED8B07C
:101AE000232A22C01CF023C01DF012001F6E010E1D
:101AF000206E000189B77FEF8DF081EF8DF0D0EF80
:101B00008DF01FC082F089958987FC0E89170F0E12
:101B1000876F010E816FF40E806F89892A0E606FC6
:101B2000320E616F010E626F000E726F000E736FE6
:101B30002A0E636F320E646F010E656F000E746FB4
:101B4000000E756F2A0E666F320E676F010E686F9A
:101B5000000E766F000E776F2A0E696F320E6A6F75
:101B6000010E6B6F000E786F000E796F1C0E6C6F9C
:101B7000320E6D6F010E6E6F000E7A6F000E7B6F6E
:101B8000EA0E1C6E320E1D6E010E1E6E07EC99F0F1
:101B900058EC99F0FBEC96F0DBEC98F0000E206E20
:101BA00020501200000E216E1DBEDBEF8DF0D9EF2C
:101BB0008DF0E1EF8DF01C6C1D1ED8B01D2A010EBA
:101BC000216E1FBEE8EF8DF0E6EF8DF0ECEF8DF0AB
:101BD0001E6C1F1ED8B01F2A1E501F10D8B4F3EF62
:101BE0008DF0F5EF8DF019EF8EF0010E206EFDEF08
:101BF0008DF0D8901E361F36202A1FAE02EF8EF0D1
:101C000004EF8EF0F9EF8DF01E501C5C1F501D5834
:101C1000D8A00DEF8EF00FEF8EF013EF8EF01E5068
:101C20001C5E1F501D5AD8901F321E32202E04EF0A
:101C30008EF02150D8B41FEF8EF021EF8EF025EFFB
:101C40008EF01C6C1D1ED8B01D2A1CC01CF01DC0BF
:101C50001DF01200000E0001DF6F000EE06F000E9D
:101C6000E16F000EE26F2050211022102310D8B433
:101C70003CEF8EF03EEF8EF074EF8EF0010EE36FCE
:101C800048EF8EF0D8902036213622362336E32BCB
:101C900023AE4DEF8EF04FEF8EF042EF8EF0D890E6
:101CA000DF37E037E137E23720501C5C21501D5808
:101CB00022501E5823501F58D8A061EF8EF063EFBA
:101CC0008EF06CEF8EF020501C5E21501D5A225079
:101CD0001E5A23501F5ADF81D890233222322132DC
:101CE0002032E32F4FEF8EF0DFC01CF0E0C01DF07C
:101CF000E1C01EF0E2C01FF01200AFEC98F0000946
:101D0000D8A485EF8EF087EF8EF08AEF8EF0040E68
:101D1000CBEF8EF000018951030B0009D8B493EF8B
:101D20008EF095EF8EF0A1EF8EF0010E016E8951CD
:101D3000030B026E0150025E89510218FC0B02185F
:101D4000896F8507D8A0860785518611D8B4ABEF77
:101D50008EF0ADEF8EF0BBEF8EF084EC99F060006A
:101D60000FF2D9FF600013F2DAFFDF6E0001834B40
:101D7000842B87EF8EF0B0EC8FF0036E84EC99F03B
:101D800060000FF2D9FF600013F2DAFFDF6E00018E
:101D9000834B842B03501200000E0001EE6F000EE7
:101DA000ED6F800EED25D96E010EEE21DA6E000E7C
:101DB000DF6EED4BEE2BEEBFE7EF8EF0EE5109E15B
:101DC0000A0EED5DD8A0E7EF8EF0E9EF8EF0D1EFCF
:101DD0008EF0800E296E010E2A6E000EE36F29C070
:101DE000E4F02AC0E5F0000EE76F070EE66F680E1C
:101DF000CBEC90F080C142F081C141F001018251F1
:101E00003F0B406E83C13FF0070E3F640AEF8FF037
:101E10000CEF8FF00EEF8FF0000E3F6E84C13EF09E
:101E200085511F0B3D6E86C13CF0000E876F000E82
:101E3000886F1200D3AE1FEF8FF0B0EF8FF000016C
:101E4000898943EF8FF06CEC99F0080E66EF8FF004
:101E50006CEC99F0070E66EF8FF00001852940ECDD
:101E600099F0040E66EF8FF0070E00018719D8B4C1
:101E70003CEF8FF03EEF8FF040EF8FF06FEC99F07A
:101E80000F0E66EF8FF072C0DFF073C0E0F002D883
:101E900054EF8FF00500FA6E6051FD6E6151FE6ED9
:101EA0006251FF6EFA501200010AD8B434EF8FF07D
:101EB000030AD8B428EF8FF0010AD8B423EF8FF0CB
:101EC000070AD8B42DEF8FF034EF8FF01200000E18
:101ED000BA6E010EBB6E800EBC6EE30EC26EC3689E
:101EE000800EC46E000E3A01606F000E506F000E3F
:101EF000406F4083000E816F0F0E516F000E416FD7
:101F0000C00E616F000E5A6F000E5B6F000E6A6F9D
:101F1000000E6B6F000E426F000E526F180E626F54
:101F2000BF0E436F53696369446954696469080E5D
:101F3000846F140EE26F260E126F210E136F220EA5
:101F4000146F0D0E156F130E166F080EC06F100E66
:101F5000D16F110ED26F170EE56F130EE16F1200E5
:101F600000018989D4EF8FF087EC99F0080EF7EF24
:101F70008FF087EC99F0070EF7EF8FF000018529BD
:101F80004AEC99F0040EF7EF8FF0070E0001871965
:101F9000D8B4CDEF8FF0CFEF8FF0D1EF8FF08AEC88
:101FA00099F00F0EF7EF8FF072C00CF073C00DF0C8
:101FB00002D8E5EF8FF00500FA6E6051FD6E6151B9
:101FC000FE6E6251FF6EFA501200010AD8B4C5EFDE
:101FD0008FF0030AD8B4B9EF8FF0010AD8B4B4EF88
:101FE0008FF0070AD8B4BEEF8FF0C5EF8FF0120064
:101FF000216E1C501D101E10D8B401EF90F003EF9D
:1020000090F024EF90F02150030D600EF324D96E70
:10201000000EF420DA6E600073F0DEFF600077F0EF
:10202000DEFF60007BF0DEFF2150020D720EF32414
:10203000D96E000EF420DA6E60007FF0DEFF6000E3
:1020400083F0DDFF3EEF90F02150030D600EF3248E
:10205000D96E000EF420DA6E2A0EDE6E320EDE6EBF
:10206000010EDE6E2150020D720EF324D96E000EA9
:10207000F420DA6E000EDE6E000EDD6E1200066ECB
:10208000015002100310D8B448EF90F04AEF90F0DE
:102090006BEF90F00650030D600EF324D96E000E26
:1020A000F420DA6E600007F0DEFF60000BF0DEFF68
:1020B00060000FF0DEFF0650020D720EF324D96EA1
:1020C000000EF420DA6E600013F0DEFF600017F0FF
:1020D000DDFF85EF90F00650030D600EF324D96EFE
:1020E000000EF420DA6E380EDE6E330EDE6E010E58
:1020F000DE6E0650020D720EF324D96E000EF4202F
:10210000DA6E000EDE6E000EDD6E12000001E85188
:10211000E911EA11EB11D8B490EF90F092EF90F042
:10212000C2EF90F0010E246E9CEF90F0D890E8374B
:10213000E937EA37EB37242AEBAFA1EF90F0A3EFB2
:1021400090F096EF90F0E851E45DE951E559EA51DD
:10215000E659EB51E759D8A0B0EF90F0B2EF90F00C
:10216000BAEF90F0E851E45FE951E55BEA51E65BD4
:10217000EB51E75BD890EB33EA33E933E833242EB5
:10218000A3EF90F0E4C0E4F0E5C0E5F0E6C0E6F0CF
:10219000E7C0E7F012000001E86FE4C0EBF0E5C033
:1021A000ECF0E6C0E9F0E7C0EAF00001E85176ECB7
:1021B0008DF00009D8B4DFEF90F0E1EF90F0D5EFAB
:1021C00090F0AE0E226E260E236E010E246EE90EE6
:1021D000256E000E266E3FEC98F0E30E1C6E000E8E
:1021E0001D6E000E1F6E010E1E6EA1EC97F0000E0C
:1021F000226E000E236E000E246E000E256E000E61
:10220000266E31EC98F054EC99F029EC97F0E80642
:10221000D8B40DEF91F00FEF91F005EF91F01200AF
:102220003901A3A716EF91F018EF91F01BEF91F091
:102230006F00A0F738F0000E2C6E000E2B6E2C50A5
:1022400009E1800E2B5CD8A028EF91F02AEF91F0E5
:102250002CEF91F038EF91F0000E2B24D96E010E87
:102260002C20DA6E000EDF6E2B4A2C2A1FEF91F025
:102270003901938D000E366E3D01F289000EF96F23
:10228000000EFA6F000E386E000E0101006F000E96
:102290002C6E000E2B6E000E2E6E000E2D6E000E9C
:1022A000386E390193871200B60EF66E300EF76E57
:1022B000010EF86E00EEC0F110EE1AF009006F008A
:1022C000D7FFEEFFE550E150F9E11E0EF66E2F0E3E
:1022D000F76E010EF86E00EEBBF010EE24F0090070
:1022E0006F00D7FFEEFFE550E150F9E100EE00F29C
:1022F000C00EEE6AE806FDE100EE00F1C00EEE6AE7
:10230000E806FDE100EE60F05B0EEE6AE806FDE136
:1023100000EE27F01C0EEE6AE806FDE1080ED56E11
:10232000000ED66E000ED76E000100EF80F00001A7
:10233000E46F000E0001E56F0001E45176EC8DF0D2
:102340000009D8B4A6EF91F0A8EF91F09CEF91F0BE
:10235000E00E226E2A0E236E010E246EE50E256E0F
:10236000000E266E3FEC98F0E30E1C6E000E1D6E04
:10237000000E1F6E010E1E6EA1EC97F0000E226E75
:10238000000E236E000E246E000E256E000E266ECB
:1023900031EC98F054EC99F029EC97F0E806D8B4B9
:1023A000D4EF91F0D6EF91F0CCEF91F00001E55130
:1023B00012000001E56F0001E55176EC8DF0000997
:1023C000D8B4E5EF91F0E7EF91F0DBEF91F06C0E10
:1023D000226E2A0E236E010E246EE40E256E000E70
:1023E000266E3FEC98F0E30E1C6E000E1D6E000E84
:1023F0001F6E010E1E6EA1EC97F0000E226E000EF5
:10240000236E000E246E000E256E000E266E31EC3B
:1024100098F054EC99F029EC97F0E806D8B413EF53
:1024200092F015EF92F00BEF92F01200000E216E79
:10243000000E206E1E501F10D8B421EF92F023EF33
:1024400092F04BEF92F0010E226E2BEF92F0D890AB
:102450001E361F36222A1FAE30EF92F032EF92F076
:1024600027EF92F0D890203621361E501C5C1F506A
:102470001D58D8A03EEF92F040EF92F045EF92F059
:102480001E501C5E1F501D5A2080D8901F321E32D5
:10249000222E32EF92F020C01CF021C01DF012005D
:1024A00009EC94F000018951030B0009D8B45BEFEB
:1024B00092F05DEF92F06AEF92F0A4EC98F00009D0
:1024C000D8B465EF92F067EF92F06AEF92F0100ED9
:1024D0000001876F00018751030D5F0EF324F66E34
:1024E000F70EF420F76EF86A000EF82202D886EF95
:1024F00092F00500FA6E0900F550FD6E0900F550E6
:10250000FE6E0900F550FF6EFA5012000001876F51
:1025100012001CC020F01DC021F091EF92F0204A63
:10252000212A600083F0D9FF600087F0DAFFDF50D6
:10253000D8A49DEF92F09FEF92F08FEF92F0A5EF6D
:1025400092F0204A212A1E4A1F2A60007BF0F6FFE3
:1025500060007FF0F7FF000EF86E600083F0D9FF97
:10256000600087F0DAFF08006F00D7FFDFFFDF5061
:10257000D8A4BDEF92F0BFEF92F0A1EF92F012005D
:1025800000018989D5EF92F087EC99F0070EF4EFFE
:1025900092F0000185294AEC99F0030EF4EF92F0D5
:1025A0008AEC99F00A0EF4EF92F072C00CF073C04E
:1025B0000DF002D8E6EF92F00500FA6E6051FD6E64
:1025C0006151FE6E6251FF6EFA501200010AD8B4DA
:1025D000D0EF92F0030AD8B4C4EF92F0060AD8B450
:1025E000C9EF92F0D0EF92F012000001E76F000106
:1025F000E75176EC8DF00009D8B401EF93F003EFCA
:1026000093F0F7EF92F0E3C01CF0E4C01DF0E5C0DA
:102610001EF0E6C01FF0A1EC97F0000E226E000E37
:10262000236E000E246E000E256E000E266E31EC19
:1026300098F054EC99F029EC97F0E806D8B423EF21
:1026400093F025EF93F01BEF93F0120068EC99F0F4
:10265000020E0001886F39EF93F023EC99F056EFEA
:1026600093F098EC99F056EF93F0FFEC98F056EF5A
:1026700093F074C00CF075C00DF020EE63F002D83A
:102680004CEF93F00500FA6EDE50FD6EDE50FE6EEC
:10269000DE50FF6EFA501200020AD8B42DEF93F00C
:1026A000010AD8B431EF93F035EF93F01200D3AEB6
:1026B0005CEF93F082EF94F0000120EE02F0DF5126
:1026C000D926E051DA226F0078FF1CF06F0074FF0A
:1026D0001DF060007FF3D9FF600083F3DAFF6F0025
:1026E00078FF1EF06F0074FF1FF0A1EC97F0000E52
:1026F000226E000E236E000E246E000E256E000E5C
:10270000266E3FEC98F0020E1200FC0E00018917B5
:10271000020E886F899594EF93F096EC99F0B1EFE3
:1027200093F00F0EB1EF93F076C00CF077C00DF080
:1027300020EE66F002D8A7EF93F00500FA6EDE50A7
:10274000FD6EDE50FE6EDE50FF6EFA501200020A81
:10275000D8B48DEF93F0010AD8B48DEF93F091EFD8
:1027600093F01200D28A000ED2BE010E1C6ED29ED1
:10277000550ED46EAA0ED46ED490000ED76E000EF5
:10278000D66E080ED56E550ED46EAA0ED46ED480B9
:102790001CB0CDEF93F0D0EF93F0D28ED1EF93F049
:1027A000D29E3901809F8399838781818385828F1F
:1027B000838383818991819584951200F6EF93F04C
:1027C0003901A3A9E6EF93F0E8EF93F0E0EF93F07F
:1027D000600073F0F6FF600077F0F7FF000EF86E10
:1027E00008006F00D7FFEAFD1C4A1D2A600073F045
:1027F000F6FF600077F0F7FF000EF86E0800F55066
:102800000009D8A406EF94F008EF94F0E0EF93F0FD
:102810001200D0EC98F00009D8B411EF94F013EF47
:1028200094F017EF94F093EC99F031EF94F0BAEC48
:1028300098F00009D8B41FEF94F021EF94F025EF41
:1028400094F08DEC99F031EF94F0C5EC98F000091C
:10285000D8B42DEF94F02FEF94F031EF94F090EC8A
:1028600099F01200000E1F6E000E1E6E4BEF94F0DA
:102870003901A3A93EEF94F040EF94F038EF94F0C3
:102880001E501C24D96E1F501D20DA6EDF503D01F2
:10289000EA6F1E4A1F2A1E501C24D96E1F501D208D
:1028A000DA6EDF50D8A457EF94F059EF94F038EF78
:1028B00094F012000001E16F010E0001E26F89B592
:1028C00064EF94F066EF94F07FEF94F08985000E4A
:1028D000E26F855140EC99F00001E151D8B473EFFB
:1028E00094F075EF94F07BEF94F0040E876F01EC99
:1028F00096F07FEF94F0030E876FE6EC97F00001FF
:10290000E251120020EE02F00C50D9260D50DA22CE
:102910006F0078FF01F06F0074FF02F0600033F089
:10292000D9FF600037F0DAFF6F0078FF03F06F0027
:1029300074FF04F0B3EC97F0000E076E000E086E03
:10294000000E096E000E0A6E000E0B6E4DEC98F034
:10295000020E12006F00D8FF14F06F00DCFF15F0BC
:102960006F00E0FF16F06F00D4FF17F002D8C4EF3D
:1029700094F00500FA6E0001A251FD6EA351FE6EA7
:10298000A451FF6EFA50120060005FF0F5FF600086
:102990005BF0F8FF600057F0F7FF600053F0F6FFC0
:1029A0001100000E3D01EC6F000EED6F000EEE6F9A
:1029B000000EEF6F000EF06F000EF16FB00EF26FB1
:1029C000800EF36F000EF46F8A0EF56F000EF66F37
:1029D000000EF76F000EF86F000EF96F000EFA6F21
:1029E000F28BF2893901939712000001E76FE7C07B
:1029F000E3F0680E97EC91F0356E0001E605D8A47F
:102A000004EF95F006EF95F016EF95F0800E1C6E32
:102A1000020E1D6E355018EC95F0800E1C6E020EE5
:102A20001D6E32EC94F0090E68EC98F035501200EF
:102A30001E6E1E380F0B300F600073F0D9FF600060
:102A400077F0DAFFDF6E20EE01F01C50D9261D5022
:102A5000DA221E500F0B300FDF6E20EE02F01C50FA
:102A6000D9261D50DA22000EDF6E1200D3AE3BEFE6
:102A700095F084EF96F0DFC01CF0E0C01DF0000E72
:102A80001F6E010E1E6EA1EC97F0000E226E000E5E
:102A9000236E000E246E000E256E000E266E3FEC97
:102AA00098F0040E1200D3AE58EF95F09CEF96F01C
:102AB000DFC01CF0E0C01DF0000E1F6E020E1E6E87
:102AC000A1EC97F0000E226E000E236E000E246E15
:102AD000000E256E000E266E3FEC98F0020E1200DE
:102AE000D3AE75EF95F0B4EF96F0DFC01CF0E0C008
:102AF0001DF0000E1F6E010E1E6EA1EC97F0000E71
:102B0000226E000E236E000E246E000E256E000E47
:102B1000266E3FEC98F0020E1200D3AE92EF95F0C5
:102B2000CCEF96F0DFC01CF0E0C01DF0000E1F6E71
:102B3000020E1E6EA1EC97F0000E226E000E236EA8
:102B4000000E246E000E256E000E266E3FEC98F0EF
:102B5000040E12006F0060FF18F00001A74BA82BB5
:102B6000E90EA75D030EA859D8A0B9EF95F0BBEF09
:102B700095F0C1EF95F0000EA86F000EA76FAF4B58
:0E2B8000B02B3901A991600063F0D8FF11005D
:102B90006F0060FF19F03901A4950001A54BA62B29
:102BA000A65109E1040EA55DD8A0D9EF95F0DBEFA1
:102BB00095F0E1EF95F0B14BB22B000EA66F000E31
:102BC000A56F600067F0D8FF1100266E26C01CF0CC
:102BD0001D6A000E1F6E0A0E1E6ED2EC8DF01CC018
:102BE00024F01DC025F026C01CF01D6A000E1F6ECB
:102BF0000A0E1E6E14EC8DF01C50100DF3502424A0
:102C00001200D3AE06EF96F012EF97F00001895153
:102C1000FC0B0209896F85058611D8A412EF96F086
:102C200014EF96F016EF96F01AEC8FF0D8800001B2
:102C300082353BEC99F0040E12003F011E991E975D
:102C40001E951E931E911E8F1E9B1F9F1F9D2195DB
:102C5000219321813901A19D919DA19B919B3F01D0
:102C60001D691C691B691F971F951F931F911200F7
:102C70001CC01EF01DC01FF0D8901F321E32D8900D
:102C80001F321E321E506D6E1CC01EF0030E1E162B
:102C9000060E1F6ED8901E361F2E4AEF96F01E505D
:102CA0006C6E12001E6E000E1D6E3A0E1E605BEF03
:102CB00096F05DEF96F067EF96F02F0E1E6463EFCF
:102CC00096F065EF96F067EF96F0010E1D6E1DC051
:102CD0001CF01C3012003D017995600073F06EFD10
:102CE000000E6C6F738B79A578EF96F07AEF96F003
:102CF00073EF96F074AB7FEF96F082EF96F0010ED3
:102D000083EF96F0000E12000CC001F00DC002F02F
:102D1000000E046E010E036EB3EC97F0000E076E0A
:102D2000000E086E000E096E000E0A6E000E0B6E8D
:102D30004DEC98F0040E12000CC001F00DC002F032
:102D4000000E046E020E036EB3EC97F0000E076ED9
:102D5000000E086E000E096E000E0A6E000E0B6E5D
:102D60004DEC98F0020E12000CC001F00DC002F004
:102D7000000E046E010E036EB3EC97F0000E076EAA
:102D8000000E086E000E096E000E0A6E000E0B6E2D
:102D90004DEC98F0020E12000CC001F00DC002F0D4
:102DA000000E046E020E036EB3EC97F0000E076E79
:102DB000000E086E000E096E000E0A6E000E0B6EFD
:102DC0004DEC98F0040E12003901A3A9EAEF96F039
:102DD000ECEF96F0E4EF96F00D0E3D01EA6F39014D
:102DE000A3A9F5EF96F0F7EF96F0EFEF96F00A0E45
:102DF0003D01EA6F12003D0173BF01EF97F003EF51
:102E000097F011EF97F0000E796F000E7A6F000EB9
:102E1000766F6C69510E3A016A6F510E6B6F3D010E
:102E2000738F120000018951FC0B0209896F85051F
:102E30008611D8A41EEF97F020EF97F022EF97F0BD
:102E4000B0EC8FF0D8800001823545EC99F0040E8B
:102E50001200010E1C6E000189B531EF97F033EFBF
:102E600097F03DEF97F08997826958EC99F014EC50
:102E700098F02AEC99F088C01CF01C5012001C50ED
:102E80001E026F00CCFF20F06F00D0FF21F01C501D
:102E90001F02F35021261D501E02F350212620C090
:102EA0001CF021C01DF012007BEC99F078EC99F039
:102EB0000009D8B45EEF97F060EF97F066EF97F0F7
:102EC000000E4AEC99F0000E45EC99F0000E12004D
:102ED000000E3F013E6F030E3F6F000E3A6F000E73
:102EE000396F000E386F000E3D6F100E3C6F620E92
:062EF0003B6F3E9F120043
:102EF8006F0060FF1BF03901A3A985EF97F087EFFA
:102F080097F08BEF97F06000DFF0EAFD372A60005A
:102F18006FF0D8FF110077F870F869F810F862F8C8
:102F280006F852F8FCF73C30304830304D3030531A
:102F38000030302F30302F303000000189A9A7EF42
:102F480097F0A9EF97F0B2EF97F01CC083F01DC07F
:102F580084F01EC085F01FC086F089991200000118
:102F680089A9B9EF97F0BBEF97F0C4EF97F001C0CC
:102F780083F002C084F003C085F004C086F089990C
:102F88001200040E3D01736F800E746F180E756F7A
:102F9800030E7B6F000E796F000E7A6F000E766F4E
:102FA8006C691200010E966E000E956E000E976EFB
:102FB8009368000E926E3901A9919981E00E946E82
:102FC800949E1200D3AEEBEF97F08EEF98F00001CD
:102FD8008951FC0B0209896F825182253BEC99F0DB
:102FE800030E1200010EA26E000EA16E080EA36E53
:102FF8009F68000E9E6E3901A791600EA06EA08E8C
:103008001200010EAE6E000EAD6E000EAF6EAB6814
:10301800000EAA6E3901A495670EAC6E9495120045
:10302800390193939395929F93913D017A917A9563
:103038007A9F7A9D7A9376937695769112003E01DF
:10304800F851F30B0409F86FF889010EF16FC28289
:103058003A0140833E01F88F120022C01CF023C0C1
:103068001DF024C01EF025C01FF026C020F0020E5F
:10307800F8EC8FF0120022C01CF023C01DF024C011
:103088001EF025C01FF026C020F0000EF8EC8FF0CF
:10309800120007C001F008C002F009C003F00AC01E
:1030A80004F00BC005F0000E3FEC90F012005AF847
:1030B80049F840F891F87EF897F88BF837F885F8D2
:1030C800F1F72EF824F81AF81C6E3901A3A96FEF4E
:1030D80098F071EF98F069EF98F0600073F0EAFDEE
:1030E8001200800E6E6E000E6D6E000E6C6E3F014B
:0A30F8005F51FC0B02095F6F12002C
:103104006F0060FF1AF03901A1910001AD4BAE2BA5
:1031140060006BF0D8FF110000018951FC0B02091B
:10312400896F8251822545EC99F0030E12003D010E
:1031340078BB9FEF98F0A2EF98F0010EA3EF98F000
:10314400000E12003D0174BBAAEF98F0ADEF98F0A9
:10315400010EAEEF98F0000E12003D0178B1B5EF0C
:1031640098F0B8EF98F0010EB9EF98F0000E120045
:103174003D0179B5C0EF98F0C3EF98F0010EC4EFAC
:1031840098F0000E12003D0176B9CBEF98F0CEEF27
:1031940098F0010ECFEF98F0000E12003D0179BFB8
:1031A400D6EF98F0D9EF98F0010EDAEF98F0000E10
:1031B4001200390193839385928F93813D017A851F
:1031C4007A8F768112003F0112511C6E13511D6ECD
:1031D40014511E6E1F6A12001F6E1FC01EF00F0EC8
:1031E4001E161E501C6E1D6A12004FEC99F0000151
:1031F4008995020E886F0F0E12004FEC99F00001B2
:103204008995000E886F0F0E12001CC0A2F01DC01D
:10321400A3F01EC0A4F01200D3AE13EF99F09AEFFE
:1032240099F0050E1200D3AE1AEF99F09CEF99F0C5
:10323400010E12007EEC99F07BEC99F030EC99F0E1
:103244001200000185514AEC99F012EC97F012003B
:103254003D01739F000E796F7885120000018995F6
:10326400000E886F0F0E12003901A191D280919146
:1032740012001C6E600073F06BFD12001C6E600087
:1032840073F06CFD1200016E600007F06BFD12001C
:10329400016E600007F06CFD12003D01739F78859C
:1032A400738F1200000E5AEC94F01200000E3D01D0
:1032B400796F12007EEC99F0090E120081EC99F0FE
:1032C400030E120081EC99F0040E1200000E3D0171
:1032D400796F12003D01738D12003D01739D120040
:1032E4003901A195110050EC92F012003D016C518E
:1032F40012003D01739B12003D01748D12003D01CB
:10330400749D12003D016A5112003D01738D12003B
:103314003D01739D12003D01799512003D0176999E
:1033240012003D01799F1200010E1200020E1200DC
:0A333400050E1200010E1200120037
:020000040020DA
:10000000FF0FFF0FFF0FFF0FFF0FFF0FFF0FFF0F80
:020000040030CA
:0A0000008CFEFFFF9FFFFFFFFFFFD4
:00000001FF
